:100000000C942A001895000018950000189500001F
:10001000189500001895000018950000189500002C
:10002000189500001895000018950000189500001C
:10003000189500001895000018950000189500000C
:1000400018950000189500001895000018950000FC
:10005000189500008FE58DBFC8E3E0E24E2E84E0E6
:100060008EBFD4E0F4E05F2EA89584B7082E877F7A
:1000700084BF88E1992781BD91BDEEEFF3E0A0E652
:10008000B0E088278D933197E9F70E94D802662463
:1000900087E886B980E087B9379A8CE00E9426030A
:1000A0000E94C30281E090E0A0E6B0E08D939C93B3
:1000B000A0E6B0E00D911C91043050E015071CF053
:1000C00011F00C94AB00A0E6B0E00D911C9141E062
:1000D00050E0041B150BA2E6B0E00D931C93A2E6C2
:1000E000B0E00D911C9144E050E0040F151FA4E610
:1000F000B0E00D931C932091600011E00E94C802B3
:10010000EEE7FCE00E94BC02A8E0B4E0E2E6F0E02A
:100110000E94D1050E94B402E2E8FCE00E94BC0209
:10012000209160001CE00E94C802EEE7FCE00E9403
:10013000BC02A8E0B4E0E4E6F0E00E94D1050E9431
:10014000B402E2E8FCE00E94BC02A0E6B0E00E943B
:100150008B020C94580080E090E0A0E6B0E08D9314
:100160009C93A0E6B0E00D911C91073050E015077C
:100170001CF011F00C94FE0007B1007E809160002D
:1001800090E0890F082707B90E944F04A0E6B0E06D
:10019000AD90BD90A6E6B0E0AA0CBB1CAA0DBB1D9D
:1001A0008D939C93EAE5FCE00E945D05E0E6F0E0BB
:1001B000A190B190E6E6F0E0AA0CBB1CEA0DFB1D95
:1001C000D190E080FF2400270E947C040E94C90493
:1001D000EDE0F0E0A0E6B0E0AD90BD90A6E7B0E0C5
:1001E000AA0CBB1CAA0CBB1CAA0DBB1D0E94270697
:1001F000A0E6B0E00E948B020C94B100E6E7F0E0CC
:100200000E945D04EEE5FCE00E9454050E941F057B
:10021000EDE0F0E0A6E7B0E00E942706EAE7F0E0B4
:100220000E945D04E2E6FCE00E9454050E941F0566
:10023000EDE0F0E0AAE7B0E00E942706EEE7F0E08C
:100240000E945D04E6E6FCE00E9454050E941F0542
:10025000EDE0F0E0AEE7B0E00E942706E2E8F0E073
:100260000E945D04EAE6FCE00E9454050E941F051E
:10027000EDE0F0E0A2E8B0E00E942706E6E8F0E05A
:100280000E945D04EEE6FCE00E9454050E941F05FA
:10029000EDE0F0E0A6E8B0E00E942706EAE8F0E032
:1002A0000E945D04E2E7FCE00E9454050E941F05E5
:1002B000EDE0F0E0AAE8B0E00E942706EEE8F0E00A
:1002C0000E945D04E6E7FCE00E9454050E941F05C1
:1002D000EDE0F0E0AEE8B0E00E942706E2E9F0E0F1
:1002E0000E945D04EAE7FCE00E9454050E941F059D
:1002F000EDE0F0E0A2E9B0E00E942706A8E0B4E05B
:10030000AF93BF93E6E7F0E00E9458040E946203B7
:1003100011E002E0BF91AF910E947305E8E0F4E0C4
:10032000A6E9B0E00E942206A8E0B4E0AF93BF9334
:10033000EAE7F0E00E9458040E94620311E001E045
:10034000BF91AF910E947305E8E0F4E0ACE9B0E042
:100350000E942206A8E0B4E0AF93BF93EEE7F0E07E
:100360000E9458040E94620311E001E0BF91AF9126
:100370000E947305E8E0F4E0A2EAB0E00E942206E1
:10038000A8E0B4E0AF93BF93E2E8F0E00E94580425
:100390000E94620311E001E0BF91AF910E947305DA
:1003A000E8E0F4E0A8EAB0E00E942206A8E0B4E0A9
:1003B000AF93BF93E6E8F0E00E9458040E94620306
:1003C00011E000E0BF91AF910E947305E8E0F4E016
:1003D000AEEAB0E00E942206A8E0B4E0AF93BF937B
:1003E000EAE8F0E00E9458040E94620311E000E095
:1003F000BF91AF910E947305E8E0F4E0A4EBB0E098
:100400000E942206A8E0B4E0AF93BF93EEE8F0E0CC
:100410000E9458040E94620311E000E0BF91AF9176
:100420000E947305E8E0F4E0AAEBB0E00E94220627
:10043000A8E0B4E0AF93BF93E2E9F0E00E94580473
:100440000E94620311E000E0BF91AF910E9473052A
:10045000E8E0F4E0A0ECB0E00E94220680E090E04A
:10046000A0E6B0E08D939C93A0E6B0E00D911C91C6
:10047000033050E015071CF011F00C948302A0E645
:10048000B0E00D911C9141E050E0040F151FA2E671
:10049000B0E00D931C93A0E6B0E00D911C9144E0F8
:1004A00050E0040F151FA4E6B0E00D931C932091BB
:1004B000620015E00E94C802A0E6B0E00D911C9118
:1004C00046E050E00E944504A6E9B0E0A00FB11F4D
:1004D0000E94B6022091620010E10E94C802A4E6C8
:1004E000B0E00D911C9146E050E00E944504A6E961
:1004F000B0E0A00FB11F0E94B602A0E6B0E00E94DB
:100500008B020C94340280E991E00E9453030C9416
:100510005200F894FFCFED91FC91EF5FFF4FFC93F9
:10052000EE93089505D00E94450400FC0CD0089578
:100530000024E89457FF02C009D0689400F80BD05B
:1005400010F80124089502D009D0089550954095DF
:100550004F5F5F4F0895E89417FF08950095109539
:100560000F5F1F4F68940895A8E0B4E08D91882331
:1005700011F066D0FBCF08950E945005802D11F038
:100580005FD0FACF089581E061D00FD080E85EC0DF
:100590008FE7213039F08FEB223021F083E92330CF
:1005A00009F083ED810F0C94260383E099277BC02B
:1005B0008AEF90E00E945303A79AA69AA59AA49A5C
:1005C000A29AA19AA99885E090E00E945303AA9864
:1005D000AF98AE98AD9AAC9AAA9AEF93FF93ECE8D5
:1005E000F1E00E944703FF91EF91AA9859D0AA9A8F
:1005F000EF93FF93ECE8F1E00E944703FF91EF9146
:10060000AA984ED0AA9AEF93FF93ECE8F1E00E94EB
:100610004703FF91EF91AA9843D0AC98AA9AEF9321
:10062000FF93ECE8F1E00E944703FF91EF91AA9855
:1006300037D088E20BD08EE009D086E007D008954D
:10064000A99A829505D004D02BD00895A998F9CF06
:10065000859510F4AC9A01C0AC98859510F4AD9ACC
:1006600001C0AD98859510F4AE9A01C0AE988595FD
:1006700010F4AF9A01C0AF98AA9AEF93FF93ECE8F9
:10068000F1E00E944703FF91EF91AA9808953197F6
:10069000F1F70895689462F80895E89462F808956F
:1006A00081E090E000C0EF93FF93EE27E82BE92B69
:1006B00031F0E0EAFFE03197F1F70197D1F7FF91D0
:1006C000EF9108958DE207FD8D938F2D881F802F68
:1006D000881F8F57082F6894F7F8802F87FF15C061
:1006E00080958395082F80E38D938EE28D93802FE4
:1006F000815228F080E38D9399279C930895442795
:100700000A95802F09F196D01FC0805230F09EE4E8
:100710009D9381E48D939D93EFCF4427DF92EF92D9
:10072000FF920F938FE1801B11F0082F83D089D0A7
:100730009EE29D930F91FF90EF90DF9044270395E9
:10074000003209F4D7CF2BD03F93E4EDF7E038E146
:100750002F2D1E2D0D2DFF24EE24DD244427000F08
:10076000111F221FA8F42F923F920E945005102CB7
:100770000E945005202C0E945005302C0E945005EC
:100780003197410DD21CE31CF01C3F902F9001C00B
:10079000339631963A9519F73F9107D0AFCFDD0CDC
:1007A000EE1CFF1C0A95D9F70895002719E058D0D0
:1007B0008F93802B11F0039501C08F911A95B9F793
:1007C000802F882309F496CF8F91805D8D930A95B1
:1007D000D9F792CF0065CD1D80B2E60E4059730760
:1007E000A0ACB90350D6DC01286BEE00943577003D
:1007F000CA9A3B0065CD1D00B2E60E005973070092
:10080000ACB90300D6DC01006BEE000035770000C8
:100810009A3B0000CD1D0000E60E000073070000AB
:10082000B9030000DC010000EE00000077000000CA
:100830003B000000F694E794D79447950A95D1F7CA
:10084000089500270DD08F9303958F2D8E298D2924
:10085000842BC1F78F91805D8D930A95D9F74CCF8A
:100860001F930F93002710E2440FDD1CEE1CFF1CAA
:10087000001F802F9AE0890B10F0082F43951A95DE
:1008800099F7802F0F911F9108950F92B801469FFD
:100890008001479F100D569F100D0F900895369AB6
:1008A0003699FECF369A3699FECF84B195B1089528
:1008B000D190E190F1900191089521913191419170
:1008C00051910895102F90E8FF0C001F0927990FF0
:1008D000F7941078652F90E8440F551F5927990F0A
:1008E0004795607800380895FF0C90E89027110F25
:1008F0009795F794092F0895102FBD2CDE2CEF2C1F
:10090000F02E11234AF4B094D094E094F0949FEF29
:10091000B91AD90AE90AF90A0EE1FF2039F4FE2CC6
:10092000ED2CDB2CBB240850C2F767C032F00A95CF
:10093000BB0CDD1CEE1CFF1CF9CF0E94A004D4CF21
:10094000B7FE089590E8B91611F4D0FE08959FEF10
:10095000D91AE90AF90A09F403950895502F2D2DA3
:100960003E2D4F2D612F08952DEC3CEC4CEC5DE3BA
:1009700066270FC09DDFF2DFDD24EE2490E8F92E1C
:100980000FE307C09ADF05C02227332740E251E476
:100990006627552351F1002381F194DF71F1162769
:1009A000005850580894050B18F407FD03C025C0E3
:1009B00007FD23C0469537952795F694E794D7947D
:1009C00022D0FF202AF0DD0CEE1CFF1C015073F03A
:1009D0009D2D969548F0DD203AF4EE202AF491E022
:1009E000D90E9927E91EF91E7FCF07C09FE7092F6F
:1009F000F92A9FEFD92EE92E0895DD24EE24FF2455
:100A00000027112708959F929924AA24BB2488E1E6
:100A1000D216E306F40628F0D21AE30AF40A089480
:100A200001C08894991CAA1CBB1CDD0CEE1CFF1C89
:100A30008A9571F7D92CEA2CFB2C9F90089542DF00
:100A4000E1F25038D1F21627005850580894051F8B
:100A500012F418F4CBCF08F0D0CF0BD0FF202AF03F
:100A6000BB0CDD1CEE1CFF1C3FCF0F5F0BF4BECF99
:100A70003BCF9F929924AA24BB24992788E1990C03
:100A8000AA1CBB1CDD1CEE1CFF1C30F4920EA31E26
:100A9000B41ED91EE91EF91E8A9589F79F90089504
:100AA000C895319600200895FBDFD02CF9DFE02CAB
:100AB000F7DFF02CF5DF002D0895F2DF202DF0DFB9
:100AC000302DEEDF402DECDF502D089599278D91CC
:100AD00093958823E1F7939511968C9311978E91B6
:100AE0009A95D1F70895EA2FFB2F00244C918D9110
:100AF00003948E32E1F711248D9113948823E1F74A
:100B00001A94101640F41197202F2119239580E391
:100B10008D932A95E9F7113039F59927AE2FBF2F1C
:100B2000A00DB91FA00FB91F8C919C93853308F4B9
:100B300021C031E08E918E32E9F38D3241F0830F86
:100B40008A3319F480E331E001C033278C93AE1768
:100B500089F7332341F0AE2FBF2FB8DF81E34D3249
:100B600009F43196808308958827E00DF81FE00F7F
:100B7000F81F80830895000F111F221F331F08954F
:100B800000951095209530950F5F1F4F2F4F3F4FC9
:100B90000895019110810EC0019111912191308130
:100BA0000BC00191108117FF05C03FEF2FEF04C06C
:100BB000008111272227332737FF03C0E1DF8DE2B1
:100BC0008D93CF93DF93CF92DF92EF92AA24BB2431
:100BD000CC24DD24EE2440E2CAE0DD2755E093E397
:100BE0008881890F87FD9F7083FD907F891B899382
:100BF0005A95A9F7C0DFAA1CBB1CCC1CDD1CEE1C3F
:100C00004A9551F7E894EFE0FF2782910ED0EB3040
:100C1000E0F71EF068948A2D0CD088278D93EF9012
:100C2000DF90CF90DF91CF910895982F829501D0DA
:100C3000892F8F70805D26F0803309F408956894C1
:100C40008D93089581918D938823E1F7089594E021
:100C500081918D939A95E1F7089500C07F4400003B
:100C6000A040000020410000C841000048420000B0
:100C7000C84200004843000096430000FA4343483E
:0A0C800000003D2020202056000057
:00000001FF
